:1000000000180020C1000000A506000071060000D5
:100010007106000071060000710600007106000004
:10002000710600007106000071060000A5060000C0
:10003000A506000071060000A5060000610600008C
:10004000A5060000A5060000A5060000A506000004
:10005000A5060000A5060000A5060000A5060000F4
:10006000A5060000A5060000A5060000A5060000E4
:10007000791900000D220000591D0000A50600009E
:10008000A5060000A5060000A5060000A5060000C4
:10009000A5060000A5060000A5060000A5060000B4
:1000A00099080000A5060000A5060000A5060000AE
:1000B000A5060000A5060000A5060000A506000094
:1000C00038B500F0F3FA444A444B1A60444A454BB1
:1000D0001A60454A454B1A60454B0822197811426F
:1000E00002D019780A431A70424B2A221A70002350
:1000F000414A42499A188A4204D24149C9580433B4
:100100001160F5E73F4B40491A1F181D00238A4232
:1001100002D21360031CF6E73C493D4A5958101CB3
:1001200099500433C02BF7D100239A083949920023
:10013000521803211940C9001568FF248C40A543BB
:100140002C1C80258D40291C214301331160202B5C
:10015000EBD1314B8A221860304B1A70304B24227D
:100160001A70304BA0221A701A1C2F4B197888076E
:10017000FBD51978CD06FCD418780C21014008294C
:10018000FAD12A49032008702949402008701978BB
:100190008806FCD519784D06FCD52649C020800577
:1001A00008602021117019780C220A400C2AFAD11B
:1001B000214A224B1A60224A224B1A60224B072204
:1001C0001A6062B600F0E8F902F002F900F074FA81
:1001D00001F078F8FEE7C046300004F034800440B7
:1001E000823F0000388004400100000F3C80044042
:1001F00002D0074000E0074060FDFF1F58FEFF1FD0
:100200001C2700005CFEFF1F5401002000000000BE
:1002100000F9FF1F00E400E008ED00E00050064098
:1002200001400640004006400640064004400640AB
:100230000540064044800440C00005050480044099
:10024000BF5D000014E000E010E000E0FFFFFFFFF2
:10025000FFFFFFFFFFFFFFFFFFFFFFFFFFFFFFFFAE
:10026000FFFFFFFFFFFFFFFFFFFFFFFFFFFFFFFF9E
:10027000FFFFFFFFFFFFFFFFFFFFFFFFFFFFFFFF8E
:10028000FFFFFFFFFFFFFFFFFFFFFFFFFFFFFFFF7E
:10029000FFFFFFFFFFFFFFFFFFFFFFFFFFFFFFFF6E
:1002A000FFFFFFFFFFFFFFFFFFFFFFFFFFFFFFFF5E
:1002B000FFFFFFFFFFFFFFFFFFFFFFFFFFFFFFFF4E
:1002C000FFFFFFFFFFFFFFFFFFFFFFFFFFFFFFFF3E
:1002D000FFFFFFFFFFFFFFFFFFFFFFFFFFFFFFFF2E
:1002E000FFFFFFFFFFFFFFFFFFFFFFFFFFFFFFFF1E
:1002F000FFFFFFFFFFFFFFFFFFFFFFFFFFFFFFFF0E
:10030000FFFFFFFFFFFFFFFFFFFFFFFFFFFFFFFFFD
:10031000FFFFFFFFFFFFFFFFFFFFFFFFFFFFFFFFED
:10032000FFFFFFFFFFFFFFFFFFFFFFFFFFFFFFFFDD
:10033000FFFFFFFFFFFFFFFFFFFFFFFFFFFFFFFFCD
:10034000FFFFFFFFFFFFFFFFFFFFFFFFFFFFFFFFBD
:10035000FFFFFFFFFFFFFFFFFFFFFFFFFFFFFFFFAD
:10036000FFFFFFFFFFFFFFFFFFFFFFFFFFFFFFFF9D
:10037000FFFFFFFFFFFFFFFFFFFFFFFFFFFFFFFF8D
:10038000FFFFFFFFFFFFFFFFFFFFFFFFFFFFFFFF7D
:10039000FFFFFFFFFFFFFFFFFFFFFFFFFFFFFFFF6D
:1003A000FFFFFFFFFFFFFFFFFFFFFFFFFFFFFFFF5D
:1003B000FFFFFFFFFFFFFFFFFFFFFFFFFFFFFFFF4D
:1003C000FFFFFFFFFFFFFFFFFFFFFFFFFFFFFFFF3D
:1003D000FFFFFFFFFFFFFFFFFFFFFFFFFFFFFFFF2D
:1003E000FFFFFFFFFFFFFFFFFFFFFFFFFFFFFFFF1D
:1003F000FFFFFFFFFFFFFFFFFFFFFFFFFFFFFFFF0D
:10040000FFFFFFFFFFFFFFFFFFFFFFFFFEFFFFFFFD
:1004100010B5064C2378002B07D1054B002B02D0DA
:10042000044800E000BF0123237010BD58FEFF1FE9
:10043000000000001C27000008B5084B002B03D06B
:100440000748084900E000BF07480368002B03D0B5
:10045000064B002B00D0984708BDC04600000000A6
:100460001C2700005CFEFF1F58FEFF1F000000005D
:1004700008B50D20012100F033F808BD10B5FA24AD
:100480000121A4000D2000F00BF8201C00F06AF8F8
:1004900000210D2000F004F8201C00F063F810BDCE
:1004A00010B51A2818D80C2358430C4A8358101832
:1004B0001C7D027A224205D0002901D01A710BE07E
:1004C0001A7209E043681A68002902D003210A431E
:1004D00001E002218A431A6010BDC0461C240000BE
:1004E00010B51A2818D80C2358430C4A14186368FE
:1004F0008258247A012904D1117D0C431475A2225B
:1005000005E0107DA0431075002902D18022520021
:1005100001E00422FF321A6010BDC0461C24000016
:1005200010B572B60B4B0C491A680C4B1B68096866
:1005300062B6480104D532219142894149425B1893
:100540000748FA24801A1821A4005C4301F0D2FE67
:10055000201810BD18E000E004ED00E074FEFF1F5D
:10056000BF5D000038B5041CFFF7DAFF051C002C46
:100570000ED0FFF7D5FF074B401B984205D9013C31
:10058000002C05D0FA239B00ED1800F043FDF0E7A6
:1005900038BDC046E70300001C4B8022D20510B5D1
:1005A0001A60802212061A60194B0020186019493F
:1005B000194B1A4A196028231360194A194C136001
:1005C000194A1360194A1360194A1360194A1360D3
:1005D00009222260184C2060184C2160184C2360BE
:1005E000184C2360184C2260184C20601848016099
:1005F00018490B6018490B60184B1A6000F0C2FCD8
:100600000420FFF7AFFF00F021FC10BD00E100E087
:1006100004800340FFBF0000088003400C800340BB
:1006200014800340008003401C800340248003406A
:100630002C80034034800340049003400890034022
:100640000C900340149003400090034004A003402A
:1006500008A003400CA0034014A0034000A00340E6
:10066000024B1A6801321A607047C04674FEFF1FC1
:1006700010B50B4C23685A0301D500F00DF923681F
:100680005A0501D501F078F923681A0501D501F062
:10069000BDFD2368DA04ECD501F05EFBE9E7C04656
:1006A0003480044008B5FFF7E3FFFFFF014B002251
:1006B0001A607047008104407047FFFFEFF313801A
:1006C000002821D1EFF31082002A1FD1EFF3058318
:1006D000002B0FD0101C0F2B0ED91A1C103A9208A9
:1006E0000B49032092000340521883401068D84001
:1006F000C0B201E080204000EFF31182002A05D053
:10070000824203D2101C01E0012040427047C046E3
:1007100000E400E0F0B50B4F02223B780A4E1A438A
:10072000D2000A4DB418606028788824002800D0D0
:10073000C82409040C43B45001225040534028708F
:100740003B70F0BDF4FEFF1F00F8FF1F7CFFFF1F92
:10075000431E10B5052B0FD872B6084A9900885869
:10076000002807D044685B008C50054A01889C5AD9
:10077000611A995262B600E0002010BDDCFEFF1F36
:1007800046010020431E0020052B09D872B6054AF9
:100790009B009B58002B02D001305B68FAE762B6E1
:1007A0007047C04638FFFF1F38B572B60123164A9E
:1007B0009A18013A127811071CD5144A5C01A55801
:1007C0009900002D05D1131908305860104BA35023
:1007D0000AE001242143C9008C58002C0AD1531887
:1007E000083058600B4B8B500B4B1A78013A1A703B
:1007F00062B608E00133072BD9D162B6064B00225E
:100800001A7000F097FB38BD7026000000F8FF1F3B
:1008100088004000C800400072FFFF1F421E10B554
:10082000052A30D8022380001843174BC0001B183C
:1008300072B6164CA05C032809D801F047FD1402DB
:1008400016050833022011E0083304200EE010489A
:10085000920014580F4B002C01D1115001E0985810
:10086000416099500EE0032000E00520A0540A1CCE
:1008700008325A608822180700D5C822098809045E
:100880000A431A6062B610BD00F8FF1F94FEFF1FF6
:1008900038FFFF1F50FFFF1FF7B5B9480478061C4B
:1008A000E4B261071DD5B74B1B78002B16D0B64AB2
:1008B0001378DBB2002B05D0013BDBB21370002BA9
:1008C00000D100BEB14A1378DBB2002B06D0013B49
:1008D000DBB21370002B01D100F0A0FEA84A042364
:1008E00013700825221C2A4000D146E2A84BA94CCF
:1008F0001B78DBB21E099A08002E00D0CFE1D5008C
:1009000065192B686A689806000F01380C2800D911
:10091000C2E101F0E5FC7F017F01C101C101C1011C
:10092000C101C101C1019E01C101C101C1010D008F
:100930001368994F526899493B6029607A609848DA
:10094000984F9949002501229BB23D602561A56120
:1009500002708B4218D8D021C9008B4200D3DFE04F
:10096000812191408B4200D1B9E006D8802B00D183
:10097000A0E0822B00D1A2E0E8E08C4A934200D1B3
:10098000BDE0A022D20014E0902109018B4215D0D5
:100990000AD8882109018B4200D0D7E0794B844CDA
:1009A0001B78161C2370D6E0824A934200D12EE1B8
:1009B000814A0026934200D1CCE0C7E0764F714BCC
:1009C000BA781A706319186A000603D5586A08388D
:1009D00000F0B0FA0835C02DF4D100252E1C774F59
:1009E000E859002805D04168019100F0A3FA019868
:1009F000F7E77851724B734FE850E859002805D05B
:100A00004268019200F096FA0198F7E76E4B6F4A40
:100A1000E8507300D0526E4B7851F05C02380328D6
:100A200007D801F053FC02040204002200E0012276
:100A30009A5501360435062ED1D1664F00233B70FE
:100A40000125654BEA18654B9200EB18013B1B78BA
:100A50001370180720D500F04FFA6B01002805D05D
:100A6000E218083050605E4AE25003E0E0503B7804
:100A700001333B7000F040FA0122AB001343DB006E
:100A8000002805D04549E21808305060E15003E0E5
:100A9000E0503B7801333B70AB0002221A43D20096
:100AA0000026A6500322134393400135E650072D3C
:100AB000C7D14FE03E4C0226257065704BE0364FA3
:100AC000BB88062B42D83A4C46489B00257065707F
:100AD0001B181B78022633423DD022703BE02E4D7E
:100AE0007F22AB881A40062A30DC6E88002E2DD17A
:100AF0003C4F9B00DB191A7802218A430EE0264DF9
:100B00007F22AB881A40062A20DC6E88002E1DD179
:100B1000344F9B00DB191A7802210A431A7019E03E
:100B20001D4D314B6A88A9885C68002C0ED018884E
:100B3000904209D15888884206D1120A032A01D16D
:100B4000267808E01E8906E00C33EDE7254B0F22DE
:100B50001A705CE0341C104FFB889E4200D91E1CAA
:100B6000371E402F00D94027201C391CFFF7D2FD2B
:100B7000E419F61B3AD1351C402F3BD047E0C04664
:100B8000802007407BFFFF1FF5FEFF1FD0FFFF1FE8
:100B90009020074000F8FF1F68FFFF1FC8004000BB
:100BA0007CFFFF1F78FEFF1F81060000020300008C
:100BB00073FFFF1F21090000210A0000DCFEFF1F58
:100BC0007CFEFF1F38FFFF1F50FFFF1F4601002064
:100BD00094FEFF1F72FFFF1F30C801107026000037
:100BE00088004000C0200740782600004025B5421C
:100BF00000D9351C201C291CFFF78CFD6419761BBD
:100C000001D1402D03D1784D784B2C601E800122FC
:100C1000774B40E0774B78491F688F4216D159686F
:100C2000764B994212D11378A92B0FD15378452BCB
:100C30000CD19378C22B09D1D3786B2B06D1704B92
:100C400000200522011C1A70FFF764FD6D4B2B601C
:100C500022E0654F3D68002D13D064480688341E9D
:100C6000402C00D94024211C281CFFF753FD361BC3
:100C70005E49B6B20E80002E01D1402C00D12E1953
:100C80003E605C4BA0221988D200914204D1002220
:100C90005A709A785C4B1A700122554B61E0D20071
:100CA000A4186068013E0838F6B22B4036D000F038
:100CB00041F95649B0004258554B002A1BD055689F
:100CC0004550111C985D0831616003280BD801F074
:100CD000FDFA02040608032104E0022102E00521D6
:100CE00000E0042199558823270700D5C8231288DE
:100CF000120413433CE0985D032808D801F0E6FA9B
:100D000039390204002200E001229A5531E02C40DA
:100D1000624262410324A41A9C552AE06288028040
:100D2000002A20D03B4D43804360B3005F593A49CD
:100D3000002F01D1585101E0CD586860C850374BA1
:100D40007600F15A5218F25200F0D6F8002804D07A
:100D50000830606020070AD507E0314B20601A7820
:100D600001321A7005E02C4201D0264B00E02D4BD9
:100D700023602D4908230B708FE5012004421ED00B
:100D80001B4902230B70294B264C1A70284B294D06
:100D90001C609C60284C1A61DC609A615D60274B86
:100DA0000D241C70264CFF232370174C33702270C7
:100DB000244A1370244B9F221A70087013E063B208
:100DC000002B04DA1D4B0D221A708023337002238E
:100DD0001C4204D01A4A1178C9B211703370102322
:100DE0001C4200D03370F7BD78FEFF1F70FFFF1F5D
:100DF0009420074068FFFF1F210900030100040041
:100E0000F5FEFF1FC80040009820074038FFFF1F75
:100E100094FEFF1FDCFEFF1F7CFEFF1F460100202B
:100E200072FFFF1F8800400080200740F4FEFF1F74
:100E300000F8FF1F9CFEFF1FF8FEFF1FC0200740A9
:100E4000882007408C2007408420074010B500F020
:100E5000E3FF00221A4B0021D1509818083241605C
:100E6000C82AF7D1174A80201468C00220431060B6
:100E7000180A154AC0B21070180C144AC0B210708B
:100E8000134A1B0E1370134AFF231370124A1348A0
:100E90001370134A13700122027012480170124934
:100EA0000A70124A116899430B1C70210B4313609E
:100EB0000F4B802252041A600E4B10221A7010BD84
:100EC00000F8FF1F348004409C200740B0200740FA
:100ED000B420074080200740882007409420074026
:100EE00010200740002107408420074018E400E05C
:100EF00000E100E00821074038B572B60B4C2568C8
:100F0000281C01F047FA0B2802D962B600200CE039
:100F100080231B06C3409D43256062B64823584387
:100F2000034B181800230360436038BD60FDFF1FAA
:100F300000FAFF1F10B5041C0E484821201A01F0CA
:100F4000D9F90B2815D80C4B1B78002B07D00B4B6D
:100F50001B78002B03D0201CFFF726FC09E072B69B
:100F60008022074B1206C240101C1A6810431860FA
:100F700062B610BD00FAFF1F72FFFF1F7BFFFF1F4D
:100F800060FDFF1F1B4B1C4A19781C4B082901D11F
:100F9000002102E00A2903D138211160132206E062
:100FA0000C2901D1342100E03C21116012221A6089
:100FB000134B1A78134B002A01D0002200E00122C3
:100FC0001A60114B1A78114B012A01D880220CE0CB
:100FD000042A01D8842208E0082A01D8852204E0E6
:100FE000102A01D8862200E087221A60084B0122CD
:100FF0001A70704764FDFF1F08B003400CB0034037
:101000007EFFFF1F20B0034065FDFF1F24B003409B
:101010007DFFFF1F10B5104C2378002B1BD101233F
:10102000237000F02BFA002801D000F032F800F015
:1010300051FC002801D000F035F901F095F80028A6
:1010400001D000F0BCF900F035FE002801D000F01E
:101050001AF90023237010BD7FFFFF1F08B500F0B1
:101060000DFA08BD08B500F0B9F908BD08B500F0E3
:10107000E3F908BD08B500F0ABFA08BD08B5081CD7
:1010800000F09CFA08BD08B5081C111C00F020FAFD
:1010900008BD7047044B00221A711A73FA21034AE3
:1010A000890099601A60704780FFFF1F6825000063
:1010B00008B50368C9B21B68984708BD08B503683E
:1010C000C9B21B68984708BD08B50368C9B21B6858
:1010D000984708BD08B50368C9B21B68984708BDA2
:1010E00008B50368C9B21B68984708BD08B503680E
:1010F000C9B21B68984708BD08B50368C9B21B6828
:10110000984708BD08B50368C9B21B68984708BD71
:1011100008B5044B4808C01801F0ECF800F09EFA3E
:1011200008BDC046C0C62D0010B5064B4808C01803
:10113000141C01F0DFF800F091FA201C00F0D4FA42
:1011400010BDC046C0C62D0008B500F0F5FA08BDB8
:1011500008B5081C00F01EFB08BD08B500F0BAFB7E
:1011600008BD08B500F0E2FB08BD08B500F0C2FB01
:1011700008BD08B500F090FB08BD08B500F0F2FB13
:1011800008BD08B500F094FB08BD08B5081C00F0C8
:1011900023FB012008BD08B5081C00F01DFB012041
:1011A00008BD10B5081C141C111C00F069FB201CA4
:1011B00010BD38B5081C0D1C00F068FE041C211C75
:1011C000281C00F05DFB201C38BDFFFF08B5044B58
:1011D0004808C01801F08EF800F02EFC08BDC0468B
:1011E00060E3160010B5064B4808C018141C01F047
:1011F00081F800F021FC201C00F066FC10BDC04608
:1012000060E3160008B500F087FC08BD08B5081CAF
:1012100000F0B0FC08BD08B500F04CFD08BD08B5F5
:1012200000F074FD08BD08B500F054FD08BD08B518
:1012300000F022FD08BD08B500F084FD08BD08B52A
:1012400000F026FD08BD08B5081C00F0B5FC012023
:1012500008BD08B5081C00F0AFFC012008BD10B5A2
:10126000081C141C111C00F0FBFC201C10BD38B520
:10127000081C0D1C00F00AFE041C211C281C00F098
:10128000EFFC201C38BD7047044B00221A711A7302
:10129000FA21034A890099601A60704790FFFF1F86
:1012A000882500007047FFFF044B00221A711A7353
:1012B000FA21034A890099601A607047A0FFFF1F56
:1012C000D825000008B5FFF7D3F8FFF7D7F8FFF7E8
:1012D000A1FEFAE708B50368C9B21B68984708BDC4
:1012E00008B50368C9B21B68984708BD08B503680C
:1012F000C9B21B68984708BD08B50368C9B21B6826
:10130000984708BD08B5044B4808C01800F0F2FF24
:1013100000F0ECFD08BDC04660E3160010B5064BBA
:101320004808C018141C00F0E5FF00F0DFFD201C89
:1013300000F024FE10BDC046C0C62D0008B500F068
:1013400045FE08BD08B5081C00F06EFE08BD08B5D6
:1013500000F00AFF08BD08B500F032FF08BD08B56F
:1013600000F012FF08BD08B500F0E0FE08BD08B5AA
:1013700000F042FF08BD08B500F0E4FE08BD08B566
:10138000081C00F073FE012008BD08B5081C00F021
:101390006DFE012008BD10B5081C141C111C00F0C6
:1013A000B9FE201C10BD38B5081C0D1C00F06EFDE8
:1013B000041C211C281C00F0ADFE201C38BD704709
:1013C000044B00221A711A73FA21034A89009960AA
:1013D0001A607047B0FFFF1F2826000070B5144B3D
:1013E0001B78002B20D0134C2368261C002B03D124
:1013F0000220FFF7ADF920602068002814D0438850
:10140000C218157A002D0BD002880133934204D301
:10141000FFF790FD0023336000E04380281C05E0C7
:10142000FFF788FD2560DAE70125684270BDC046F8
:101430007BFFFF1FCCFFFF1F38B50E4B1B78002B27
:1014400013D00D4C2368002B03D10220FFF780F945
:1014500020602068002808D04388C3181D7A002D1A
:1014600006D1FFF767FD2560E7E70120404200E075
:10147000281C38BD7BFFFF1FCCFFFF1F38B5124D66
:101480002B68002B04D0286800240288438811E0D0
:101490000E4B1B78002B03D00220FFF759F9286070
:1014A0002C68002CEFD10DE0C1180919097A002928
:1014B00003D00134E1189142F6DB002C02D1FFF792
:1014C00039FD2C60201C38BDCCFFFF1F7BFFFF1FA8
:1014D000F7B5344D0123071C0C1C2B70002C5DD07C
:1014E000314E306800282BD1304A0192304B1B78A6
:1014F000DBB2002B1AD00120FFF744F9052806D9EA
:10150000019B2C4A013B0193002B09D10BE00123E5
:101510002B70FFF7F1FC244A10600028F0D00FE098
:101520001378002B06D001231370002301202B70A9
:10153000404235E02B70FFF76DFD01232B70D5E79E
:101540001C4B002231681A704B884020C01A00944E
:10155000844200D90090181C0830081801900098A7
:101560001B184B80241A0023009A934204D0FA5C83
:101570000198C2540133F7E74A88FF180E4B3F2AFF
:1015800002D805221A70A9E7402200200A801870AC
:101590000120FFF743F9002232609FE72C70201CE6
:1015A000FEBDC046C0FFFF1FC4FFFF1FB51E0000E9
:1015B0007BFFFF1FC8FFFF1FD0FFFF1F07B56B4654
:1015C000D8710733181C0121FFF782FF0EBDFFFF02
:1015D00038B50F4B1B78002B19D00E4C2168002911
:1015E00015D04A88002A12D00B480023037098189F
:1015F0003F2805DC8818C018002505720133F6E77E
:1016000040230B800120FFF709F90023236038BD38
:101610007BFFFF1FC4FFFF1FD0FFFF1F38B50D4B1F
:101620001B78DBB2002B13D10B480168041C4A88DD
:1016300098183F2805DC8818C0180025057201336A
:10164000F6E740230B800120FFF7E8F80023236032
:1016500038BDC046C0FFFF1FC4FFFF1F164B8022CE
:101660001968D2000A431A60144A00231370144AFE
:1016700014491370144A1370144A1370144A1370E7
:10168000144A1160144AD12189001160134AC1041F
:10169000C90EC0B21170507093702C23D370104BD0
:1016A000FF22196891430A1C40210A431A600D4B1E
:1016B000802252011A607047348004405400002098
:1016C000D2FFFF1F130300005C0000205500002024
:1016D000D1FFFF1F40A0044044A0044000A00640EA
:1016E0000CE400E000E100E010B5124B1322997801
:1016F0009143032202400A43410701D510210A43C6
:101700009A700F220B490240042A03D18A7940249F
:1017100022438A715A7910218A43084200D00A4331
:101720005A719A7910218A43840600D50A439A7126
:1017300010BDC04600A0064008B50E4B1B685A05F8
:1017400017D50D4B1B78DBB2002B02D0FFF762FCE4
:10175000F7E70A4A802149011160094A0949D37013
:101760000422FF320A6008490A60084A1370084AD6
:10177000137008BD34800440D1FFFF1F80E100E0FA
:1017800000A0064040A0044044A0044054000020B3
:10179000D2FFFF1F38B5041C0B4B1D78EDB2002D96
:1017A000FAD1201C0121FEF79BFE291C201CFEF70C
:1017B00077FE0C225443054B054AE1581C19116071
:1017C000044B227A1A7038BDD1FFFF1F1C24000081
:1017D0005800002053000020F8B5214B071C1B685F
:1017E0005A053BD51F4B1B68002B02D01E4A1278AE
:1017F0001A711E4E002334783F220134A2425B410D
:101800005B421C401A4D2B78A3421CD1FEF756FFB9
:10181000402813DC174A13795BB2002BF2DA2B78DD
:10182000002101333F209842494149420B4012496F
:10183000C95CDBB2C9B2D1712B70E3E7FF28E1DDEF
:10184000FFF7E8FBDEE70C4BFFB21F550B4B012205
:101850001A70084BE4B2AC223470DA70F8BDC0469E
:101860003480044058000020530000205C00002019
:101870005500002000A00640D3FFFF1FD1FFFF1F2F
:1018800038B5041C4518AC4204D02078FFF7A4FFFB
:101890000134F8E738BDFFFF08B5044B1B78002B77
:1018A00002D0FFF7B7FBF8E708BDC046D1FFFF1F26
:1018B000064B074A1B781078DBB2C0B2834201D3D3
:1018C0003F3000E00138C01A7047C0465C0000207D
:1018D00055000020054B1878054BC0B21B78DBB2D1
:1018E000984200D24030C01A7047C04654000020D1
:1018F000D2FFFF1F0A4B0B4A19781378DBB29942CB
:101900000BD001333F2000219842494149420B400E
:101910000549C85CDBB2137001E00120404270470A
:1019200054000020D2FFFF1F130000200A4B1A783A
:101930000A4B1B78DBB29A420AD0013300223F21C6
:101940009942524152421340054AD05CC0B201E074
:10195000012040427047C04654000020D2FFFF1FC4
:1019600013000020024B1A78024BD2B21A70704753
:10197000D2FFFF1F5400002030B5254A1379990685
:1019800012D52449D4790B78002001333F259D429C
:101990004041404203402048E4B20078834203D0F3
:1019A0001E48C454DBB20B70D178194CC9B24BB28B
:1019B000002B1ADA23795BB2002B16DA184B194880
:1019C0001D780378DBB29D4202D16C23E3700CE0FA
:1019D000013300243F259D42644164422340124C60
:1019E000E45CDBB2E4B2D4710370402319420ED040
:1019F000117919420BD00D4B002119700C4B1B684B
:101A00008B4202D00B49097819722C23D37030BD58
:101A100000A0064054000020D2FFFF1F130000204A
:101A20005C00002055000020D3FFFF1FD1FFFF1FE7
:101A30005800002053000020164B802219685201E4
:101A40000A431A60144A00231370144A144913708D
:101A5000144A1370144A1370144A1370144A116014
:101A6000144AD12189001160134AC104C90EC0B2C1
:101A70001170507093702C23D370104B104A19685A
:101A80000A408021C9030A431A600E4B8022D2010A
:101A90001A60704734800440C80000205E000020B7
:101AA00013030000D0000020C90000205D000020CA
:101AB00008C004400CC0044000C006400CE400E034
:101AC000FFFF00FF00E100E010B5124B13229978F0
:101AD0009143032202400A43410701D510210A43E2
:101AE0009A700F220B490240042A03D18A794024BC
:101AF00022438A715A7910218A43084200D00A434E
:101B00005A719A7910218A43840600D50A439A7142
:101B100010BDC04600C0064008B50E4B1B68DA0475
:101B200017D50D4B1B78DBB2002B02D0FFF772FAF2
:101B3000F7E70A4A8021C9011160094A0949D370AF
:101B40000422FF320A6008490A60084A1370084AF2
:101B5000137008BD348004405D00002080E100E087
:101B600000C0064008C004400CC00440C80000206B
:101B70005E00002038B5041C0B4B1D78EDB2002D23
:101B8000FAD1201C0121FEF7ABFC291C201CFEF71A
:101B900087FC0C225443054B054AE1581C1911607F
:101BA000044B227A1A7038BD5D0000201C2400000E
:101BB000CC000020C7000020F8B5214B071C1B6893
:101BC000DA043BD51F4B1B68002B02D01E4A12784B
:101BD0001A711E4E0023347827220134A2425B4141
:101BE0005B421C401A4D2B78A3421CD1FEF766FDC8
:101BF000402813DC174A13795BB2002BF2DA2B78FA
:101C00000021013327209842494149420B401249A3
:101C1000C95CDBB2C9B2D1712B70E3E7FF28E1DD0B
:101C2000FFF7F8F9DEE70C4BFFB21F550B4B012213
:101C30001A70084BE4B2AC223470DA70F8BDC046BA
:101C400034800440CC000020C7000020D0000020D9
:101C5000C900002000C006405F0000205D00002099
:101C600038B5041C4518AC4204D02078FFF7A4FF17
:101C70000134F8E738BDFFFF08B5044B1B78002B93
:101C800002D0FFF7C7F9F8E708BDC0465D000020A5
:101C9000064B074A1B781078DBB2C0B2834201D3EF
:101CA000273000E00138C01A7047C046D00000203D
:101CB000C9000020054B1878054BC0B21B78DBB279
:101CC000984200D24030C01A7047C046C800002079
:101CD0005E0000200A4B0B4A19781378DBB2994258
:101CE0000BD001333F2000219842494149420B402B
:101CF0000549C85CDBB2137001E001204042704727
:101D0000C80000205E000020870000200A4B1A78DF
:101D10000A4B1B78DBB29A420AD0013300223F21E2
:101D20009942524152421340054AD05CC0B201E090
:101D3000012040427047C046C80000205E000020DD
:101D400087000020024B1A78024BD2B21A707047FB
:101D50005E000020C800002030B5254A137999069E
:101D600012D52449D4790B78002001333F259D42B8
:101D70004041404203402048E4B20078834203D00F
:101D80001E48C454DBB20B70D178194CC9B24BB2A7
:101D9000002B1ADA23795BB2002B16DA184B19489C
:101DA0001D780378DBB29D4202D16C23E3700CE016
:101DB0000133002427259D42644164422340124C94
:101DC000E45CDBB2E4B2D4710370402319420ED05C
:101DD000117919420BD00D4B002119700C4B1B6867
:101DE0008B4202D00B49097819722C23D37030BD75
:101DF00000C00640C80000205E00002087000020D0
:101E0000D0000020C90000205F0000205D000020FD
:101E1000CC000020C70000201FB572B6154B702201
:101E20001A70154A41211170144A0F211170802235
:101E30001A701A7852B2002AFBDA114B186862B68F
:101E4000104B984201D80A23584301AC211C0A22A6
:101E500000F025F80023E15C0B4A002905D058006A
:101E60001018013341800A2BF5D101335B00137048
:101E70001FBDC046000002400700024006000240AD
:101E8000080002407F96980040FEFF1F021C031CC2
:101E9000981A0133591E09780029F9D17047F8B50D
:101EA000061C0D1C171C0024301C391C00F066FA9F
:101EB000092901D8303100E03731C9B22955301C29
:101EC000391C00F017FA061E01D00134ECE72B197B
:101ED00058702B1C5A1BA24206DA1A78295D197019
:101EE0002A550133013CF5E7281CF8BD164B80222A
:101EF000196812010A431A60144A00231370144A25
:101F000014491370144A1370144A1370144A13704E
:101F1000144A1160144AD12189001160134AC10486
:101F2000C90EC0B21170507093702C23D370104B37
:101F3000104A19680A408021C9010A431A600E4BF1
:101F4000802292011A607047348004403C010020D6
:101F5000D200002013030000440100203D010020B6
:101F6000D10000200CB0044010B0044000B0064086
:101F70000CE400E0FF00FFFF00E100E010B5124BB1
:101F8000132299789143032202400A43410701D565
:101F900010210A439A700F220B490240042A03D1F0
:101FA0008A79402422438A715A7910218A4308424F
:101FB00000D00A435A719A7910218A43840600D5C9
:101FC0000A439A7110BDC04600B0064008B50E4BDA
:101FD0001B681A0517D50D4B1B78DBB2002B02D0FE
:101FE000FFF718F8F7E70A4A802189011160094ACA
:101FF0000949D3700422FF320A6008490A60084A7E
:102000001370084A137008BD34800440D1000020CA
:1020100080E100E000B006400CB0044010B0044085
:102020003C010020D200002038B5041C0B4B1D7869
:10203000EDB2002DFAD1201C0121FEF751FA291C26
:10204000201CFEF72DFA0C225443054B054AE1589B
:102050001C191160044B227A1A7038BDD10000207F
:102060001C240000400100203B010020F8B5214B5A
:10207000071C1B681A053BD51F4B1B68002B02D0A1
:102080001E4A12781A711E4E00233478272201341A
:10209000A2425B415B421C401A4D2B78A3421CD1EB
:1020A000FEF70CFB402813DC174A13795BB2002BB8
:1020B000F2DA2B7800210133272098424941494226
:1020C0000B401249C95CDBB2C9B2D1712B70E3E796
:1020D000FF28E1DDFEF79EFFDEE70C4BFFB21F5548
:1020E0000B4B01221A70084BE4B2AC223470DA7048
:1020F000F8BDC04634800440400100203B01002070
:10210000440100203D01002000B00640D300002023
:10211000D100002038B5041C4518AC4204D020780A
:10212000FFF7A4FF0134F8E738BDFFFF08B5044B03
:102130001B78002B02D0FEF76DFFF8E708BDC04604
:10214000D1000020064B074A1B781078DBB2C0B2E2
:10215000834201D3273000E00138C01A7047C046DF
:10216000440100203D010020054B1878054BC0B20A
:102170001B78DBB2984200D24030C01A7047C0468C
:102180003C010020D20000200A4B0B4A197813783A
:10219000DBB299420BD001333F20002198424941E4
:1021A00049420B400549C85CDBB2137001E00120D5
:1021B000404270473C010020D2000020FB0000207C
:1021C0000A4B1A780A4B1B78DBB29A420AD00133C9
:1021D00000223F219942524152421340054AD05CAD
:1021E000C0B201E0012040427047C0463C010020DF
:1021F000D2000020FB000020024B1A78024BD2B222
:102200001A707047D20000203C01002030B5254AEA
:102210001379990612D52449D4790B78002001331B
:102220003F259D424041404203402048E4B20078AF
:10223000834203D01E48C454DBB20B70D178194CD2
:10224000C9B24BB2002B1ADA23795BB2002B16DA33
:10225000184B19481D780378DBB29D4202D16C23DC
:10226000E3700CE00133002427259D426441644261
:102270002340124CE45CDBB2E4B2D471037040231F
:1022800019420ED0117919420BD00D4B0021197053
:102290000C4B1B688B4202D00B49097819722C2316
:1022A000D37030BD00B006403C010020D2000020B9
:1022B000FB000020440100203D010020D30000204D
:1022C000D1000020400100203B01002002B47146F3
:1022D00049084900095C49008E4402BC7047C04669
:1022E00003B47146490840004900095A49008E4428
:1022F00003BC7047002934D00123002210B4884267
:102300002CD301242407A14204D2814202D2090124
:102310001B01F8E7E400A14204D2814202D2490045
:102320005B00F8E7884201D3401A1A434C08A042E8
:1023300002D3001B5C0822438C08A04202D3001B7E
:102340009C082243CC08A04202D3001BDC08224395
:10235000002803D01B0901D00909E3E7101C10BCB9
:102360007047002801D00020C04307B4024802A1F2
:102370004018029003BDC046190000000029F0D0AB
:1023800003B5FFF7B9FF0EBC4243891A1847C04690
:102390007047C0461C2101231B04984201D3000C46
:1023A00010391B0A984201D3000A08391B099842C8
:1023B00001D30009043902A2105C40187047C046DE
:1023C00004030202010101010000000000000000FE
:1023D00070B50E4B0E4D0024ED1AAD101E1CAC4214
:1023E00004D0A300F35898470134F8E700F086F9C9
:1023F000084B094D0024ED1AAD101E1CAC4204D050
:10240000A300F35898470134F8E770BD082700008F
:1024100008270000082700001C270000420000F8E1
:1024200040A0044001000000420000F844A0044025
:1024300002000000C00000F800C0044001000000DD
:10244000000000F80490044002000000000000F8C2
:102450000890044004000000C00000F81CC00440C4
:1024600080000000C00000F810C004401000000010
:10247000C00000F808C0044004000000C00000F8DC
:102480000CC0044008000000800000F80CB00440BC
:1024900008000000800000F810B0044010000000A8
:1024A000800000F818B0044040000000800000F8F0
:1024B0001CB0044080000000800000F814B004400C
:1024C00020000000C00000F804C00440020000002A
:1024D000800000F800B0044001000000400000F857
:1024E00000A0044001000000400000F804A00440E7
:1024F00002000000400000F80CA0044008000000AA
:10250000400000F808A0044004000000C00000F8EB
:1025100014C0044020000000C00000F818C00440AF
:1025200040000000800000F804B0044002000000F9
:10253000800000F808B0044004000000020100F828
:1025400050D0044010000000020100F854D00440B4
:1025500020000000030100F878D004404000000093
:1025600000000000000000007D1000008710000047
:102570005D100000651000006D1000007510000077
:102580000000000000000000471200005F12000081
:1025900017120000271200001F1200002F12000067
:1025A000CD110000E5110000051200000D12000021
:1025B000371200003F120000E1100000ED10000093
:1025C000F9100000051100006F1200005312000006
:1025D00000000000000000008B110000A3110000AB
:1025E0005B1100006B11000063110000731100000B
:1025F00011110000291100004911000051110000C3
:102600007B11000083110000B1100000BD1000001C
:10261000C9100000D5100000B31100009711000090
:1026200000000000000000007F130000971300006E
:102630004F1300005F1300005713000067130000E2
:10264000051300001D1300003D130000451300009A
:102650006F13000077130000D5120000E112000094
:10266000ED120000F9120000A71300008B13000008
:10267000151915190000FFFF0001000066FDFF1F7E
:10268000120000000002000090FDFF1F4900000042
:1026900000220100D9FDFF1F2100000000210100E0
:1026A000C2FDFF1F0900000000220000FAFDFF1F0D
:1026B0001C00000000210000A2FDFF1F0900000017
:1026C000000300003CFEFF1F00000000010309049E
:1026D00078FDFF1F000000000203090416FEFF1F23
:1026E000000000000303090440FEFF1F000000007B
:1026F000000000000000000000000000F8B5C04627
:10270000F8BC08BC9E4670473904000095100000D4
:0C27100089120000A9120000C113000093
:10271C00FFFFFFFF0A041201000200000040C01678
:10272C0086040001010203011803540065006500D2
:10273C006E00730079006400750069006E006F0014
:10274C0009024900020100C0320904000002030022
:10275C000000092111010001221C00070583034020
:10276C0000010705040340000109040100020300F5
:10277C0000000921110100012221000705810340FD
:10278C0000010705020320000206C9FF0904A15C31
:10279C007508150026FF00954009758102952009E2
:1027AC0076910295040976B102C006ABFF0A0002CD
:1027BC00A1017508150026FF0095400901810295BD
:1027CC004009029102C026035400650065006E00AA
:1027DC00730079006400750069006E006F002000C2
:1027EC0052006100770048004900440004030904CA
:1027FC000C030000000000000000000000000000BE
:08280C000000000000000000C4
:00000001FF
